:2000000053C077C076C075C074C073C072C071C070C058C86EC06DC06CC06BC06AC069C00C
:2000200068C0A5C566C015C72CC72BC728C729C70EC727C726C725C7FDC623C722C711C75E
:200040001CC719C71EC71DC71CC713C700000000000000000003040600000000000000004A
:200060000102040810204080010204081020010204081020040404040404040402020202DB
:20008000020203030303030300000000360033003000000000003800350032000000000012
:2000A000370034003100E80411241FBECFE5D4E0DEBFCDBF10E0A0E6B0E0E6E0F4E102C0B2
:2000C00005900D92A43AB107D9F721E0A4EAB0E001C01D92A037B207E1F710E0C8EAD0E03D
:2000E00003C02297FE0189D9C63AD107D1F745D988C986CFCF93C82F80FF02C061E001C023
:2001000060E080917C00DBD8C1FF02C061E001C060E080917A00D3D8C2FF02C061E001C0E0
:2001200060E080917800CBD8C3FF02C061E001C060E080917600C3D8CF910895CF93C82F15
:2001400080FF02C061E001C060E080917400B7D8C1FF02C061E001C060E080917200AFD83A
:20016000C2FF02C061E001C060E080917000A7D8C3FF02C061E001C060E080916E009FD8FE
:20018000CF910895CF93C82F80FF02C061E001C060E080916C0093D8C1FF02C061E001C01A
:2001A00060E080916A008BD8C2FF02C061E001C060E08091680083D8C3FF02C061E001C002
:2001C00060E0809166007BD8CF910895CF93C82F80FF02C061E001C060E0809164006FD880
:2001E000C1FF02C061E001C060E08091620067D8CF910895CF93DF9300D000D000D0CDB7C4
:20020000DEB787EA90E05DD386EA90E052D686EA90E0B4D681110AC04EE750E067E870E066
:20022000CE010196E8D5CE01019648D660E080E00DD860E081E00AD861E080917C0006D863
:2002400061E080917A0002D861E080917800FED761E080917600FAD761E080917400F6D72D
:2002600061E080917200F2D761E080917000EED761E080916E00EAD761E080916C00E6D76E
:2002800061E080916A00E2D761E080916800DED761E080916600DAD761E080916400D6D7AE
:2002A00061E080916200D2D761E080916000CED760E080917C0003D860E080917A00FFD741
:2002C00060E080917800FBD760E080917600F7D760E080917400F3D760E080917200EFD7D6
:2002E00060E080917000EBD760E080916E00E7D760E080916C00E3D760E080916A00DFD716
:2003000060E080916800DBD760E080916600D7D760E080916400D3D760E080916200CFD755
:2003200060E080916000CBD780E090E04FDF80E090E028DF80E090E001DF80E090E0DADE5D
:20034000CE0101963FD664EF71E080E090E028D726960FB6F894DEBF0FBECDBFDF91CF91DC
:2003600008952F923F924F925F926F927F928F929F92AF92BF92CF92DF92EF92FF920F9300
:200380001F93CF93DF93CDB7DEB72C970FB6F894DEBF0FBECDBFCE01079614D6EB84F12CD2
:2003A0000A8510E06884712C8984912CAF80B12C80E3A81A88EFB80A64EF71E080E090E08D
:2003C000EFD624E6422E512C3AE0C32ED12C81E0ABD7892BB1F566E970E080E090E0E0D6F7
:2003E00061E0809160006BD766E970E080E090E0D7D660E08091600062D780E095D701979F
:2004000071F48FEFE81AF80A8CE3E816F10411F4E12CF12C64E670E080E090E0C1D680E003
:2004200090E0D4DE80E090E0ADDEC701B201D0D7B601CED7CB0182DEC701B601C9D75ADE3E
:20044000C6CF64EF71E080E090E0AAD684E6482E512C9AE0C92ED12C81E066D7892BA1F560
:2004600066E970E080E090E09BD661E08091600026D766E970E080E090E092D660E08091C5
:2004800060001DD780E050D7019761F40F5F1F4F0831110511F400E010E064E670E080E09A
:2004A00090E07ED680E090E025DE80E090E046DEC801B2018DD7B6018BD7CB0187DEC801BE
:2004C000B60186D75FDEC8CF64EF71E080E090E067D6B4E64B2E512C1AE0C12ED12C81E0AC
:2004E00023D7892BB9F566E970E080E090E058D661E080916000E3D666E970E080E090E029
:200500004FD660E080916000DAD680E00DD7019779F48FEF881A980A80E28816910419F4A8
:2005200088248394912C64E670E080E090E038D680E090E0DFDD80E090E000DEC401B20111
:2005400047D7B60145D7CB0141DEC401B60140D719DEC5CF64EF71E080E090E021D6E4E66C
:200560004E2E512CFAE0CF2ED12C81E0DDD6892BB9F566E970E080E090E012D661E080918F
:2005800060009DD666E970E080E090E009D660E08091600094D680E0C7D6019779F48FEF9F
:2005A000681A780A8DE06816710419F466246394712C64E670E080E090E0F2D580E090E0AB
:2005C000E1DD80E090E002DEC301B20101D7B601FFD6CB01B3DDC301B601FAD68BDDC5CF2F
:2005E00064EF71E080E090E0DBD548EE242E43E0342E54E6452E512C6AE0C62ED12C81E004
:2006000093D6892B09F046C066E970E080E090E0C7D561E08091600052D666E970E080E0DA
:2006200090E0BED560E08091600049D680E07CD6019789F48FEFA81AB80A84EEA81687E087
:20064000B80621F43BEDA32E37E0B32E64E670E080E090E0A5D561E08091600030D6C50174
:2006600060E177E2B5D6B101B3D6CB01AFDDC501B101AED6B201ACD6CB0184DDC501B201EB
:20068000A7D6B601A5D6CB0159DDC501B601A0D631DDB5CFC12C282D462DB501CE01019653
:2006A00096D3CE0101960AD468EE73E080E090E077D52C960FB6F894DEBF0FBECDBFDF914F
:2006C000CF911F910F91FF90EF90DF90CF90BF90AF909F908F907F906F905F904F903F9007
:2006E0002F9008950F931F93CF93DF9300D000D000D0CDB7DEB781E017D6019731F464E698
:2007000070E080E090E04CD52CDE64EF71E080E090E046D58091A4009091A500892B39F4A3
:2007200081E090E09093A5008093A40004C01092A5001092A4006091A40080916000BFD57E
:20074000CE0101963FD48C8104E6602F21D6892F1AE0612F1DD690E039DD8C81612F18D65D
:20076000892F90E00FDD8D81602F12D6892F612F0FD690E0E3DC8D81612F0AD6892F90E0DE
:20078000B9DC26960FB6F894DEBF0FBECDBFDF91CF911F910F9108958091D70090E02091FB
:2007A000D800821B910908952091D8008091D700281750F4E22FF0E0E752FF4F808190E0C0
:2007C0002F5F2093D80008958FEF9FEF0895E091D8008091D700E81730F4F0E0E752FF4F0F
:2007E000808190E008958FEF9FEF08950895CF92DF92EF92FF920F931F93CF93DF937C011C
:20080000CB018A012091B300222389F0EB016B01C40ED51ECC15DD0561F06991D701ED91DE
:20082000FC910190F081E02DC7010995F3CF642F78D1C801DF91CF911F910F91FF90EF9021
:20084000DF90CF900895CF93DF931F92CDB7DEB769832091B3002223D1F02091B400203282
:2008600040F021E030E0FC013383228380E090E014C08091B500E82FF0E0EA54FF4F9981E8
:2008800090838F5F8093B5008093B40004C061E0CE01019646D181E090E00F90DF91CF9106
:2008A0000895FC011382128248EE53E060E070E0448355836683778387E990E09183808303
:2008C00008951092D8001092D7001092B5001092B40081C081E08093B3006093D600109208
:2008E000B5001092B4000895F5CF0F93062F21E04091B40066EB70E08091D600C1D0109274
:20090000B5001092B4001092B3000F9108958F929F92AF92BF92CF92DF92EF92FF920F93D0
:200920001F93CF93DF93EC01F62ED42E48015901EE2009F1CFDF1E2D143008F013E01150EA
:20094000B8F0E881F98128E0129FB0011124A501940104C056954795379527956A95D2F757
:20096000CA01B9010190F081E02DCE010995E7CF60E0CE01BADF4D2D413208F040E22C2DB8
:2009800069ED70E08F2D3BD01092D8008093D700DF91CF911F910F91FF90EF90DF90CF908A
:2009A000BF90AF909F908F900895CF92EF920F931F93C22EE12C00E010E09801A8DF1F91EB
:2009C0000F91EF90CF90089521E0EFCF61E08DCF87EA90E066CF1092660181E080936401A8
:2009E0001092630161E082E16AD461E083E167D40898099880E280B985E486BF0895413295
:200A0000E8F5909166019111FCCF91E090936601209364012FEF2093F90010923E01240F13
:200A200020933D019093650190916501880F892B8093650180916301813039F41092630198
:200A40008091650183B985EC01C085EE86BF809166018130E1F380913E01841710F440913C
:200A60003E012FE331E0FB01D9018A2F821B841718F48D918193F9CF842F089580E00895FA
:200A80000F93413208F044C0909166019111FCCF92E090936601009364019FEF9093F900B2
:200AA00010923E0140933D01FB016FE371E0DB019A2F961B941718F491919D93F9CF1092DC
:200AC000650190916501880F892B8093650180916301813039F4109263018091650183B959
:200AE00085EC01C085EE86BF222321F0809166018230E1F38091F9008F3F61F08091F90085
:200B0000803251F08091F900803341F483E007C081E005C080E003C082E001C084E00F9156
:200B20000895613298F420916601243089F460931B01FC018DE191E0DC012A2F281B26176F
:200B400018F421912D93F9CF80E0089581E0089582E0089585ED86BF06B604FCFDCF109274
:200B60006601089585EC86BF1092660108951F920F920FB60F9211242F933F934F935F93C0
:200B80006F937F938F939F93AF93BF93EF93FF9381B1887F803609F499C068F5883209F4EC
:200BA0005BC090F4803109F454C038F4882309F4ECC0883009F44DC0EBC0883109F44CC025
:200BC000803209F45CC0E4C0803409F466C048F4803309F454C0883309F0DAC08093F90075
:200BE000A3C0803509F44EC0883509F45BC0883409F0CEC0CCC0883909F4BFC0A8F4883796
:200C000009F464C038F4883609F460C0803709F45DC0BEC0883809F4B0C0803909F45CC05E
:200C2000803809F0B5C058C0803B09F47FC038F4803A09F462C0883A09F478C0A9C0803C5E
:200C400009F49EC0883C09F49BC0883B09F483C09FC08091650110C090913E0180913D01C5
:200C6000981758F5E0913E0181E08E0F80933E01F0E0E15CFE4F808183B985EC7FC080931E
:200C8000F90085C0E0913E0181E08E0F80933E0183B1F0E0E15CFE4F808390913E01809114
:200CA0003D0168C0E0913E0181E08E0F80933E0183B1F0E0E15CFE4F808380916401811135
:200CC00066C081E08093630184EA5BC083E0809366011092FA00D1CF8091FA00803208F0BF
:200CE0004CC0E091FA0081E08E0F8093FA0083B1F0E0E550FF4F8083C0CF8091FA0080329C
:200D000030F4E091FA00F0E0E550FF4F108222DF6091FA0070E0E0915F01F09160018BEFF6
:200D200090E009951092FA001DDF32C084E08093660110921C0110921B01E0916101F0916C
:200D40006201099580911B01811105C081E080931B0110921D01E0911C0181E08E0F80931F
:200D60001C01F0E0E35EFE4F808183B990911C0180911B01981708F480CF85E886BF08C0DC
:200D800085EC86BF1092660103C01092F900E2DEFF91EF91BF91AF919F918F917F916F9176
:200DA0005F914F913F912F910F900FBE0F901F901895FC01208120532A3008F020E0FC010C
:200DC00081818053FAE02F9F800D11240895CF92EF920F93FC01603D87E0780710F0605D76
:200DE00077406083418322830383E482C5820F91EF90CF900895CF92DF92EF92FF920F931C
:200E00001F93CF93DF93EC017B016A01CB010996D0DF8883F7010081112707FD1095212FA9
:200E2000312FF801E154F109E331F10550F5ED5EFF4F0994F7018181813639F082818E3604
:200E400011F486E01DC087E01BC081E019C082E017C0F7018281823711F484E011C088E03F
:200E60000FC0F7018281823711F483E009C085E007C089E005C08AE003C08BE001C08CE09F
:200E80008983C701049695DF8A83C60192DF8B83C60103968EDF8C83C60106968ADF8D8365
:200EA000DF91CF911F910F91FF90EF90DF90CF90089587EA90E005DD81E008951F93CF93C4
:200EC000DF93EC0168E670E087EA90E00DDD60E087EA90E0B8DC2D811AE0822F612F58D282
:200EE000682F660F680F660F620F87EA90E0ABDC2C81822F612F4CD2682F660F680F660F1D
:200F0000620F87EA90E09FDC2B81822F612F40D2682F660F680F660F620F87EA90E093DC4C
:200F200060E087EA90E08FDC2A81822F612F30D2682F660F680F660F620F87EA90E083DC8E
:200F40002981822F612F24D2682F660F680F660F620F87EA90E077DC2881822F612F18D23F
:200F6000682F660F680F660F620F87EA90E06BDC87EA90E0DF91CF911F9128CDCF93DF93B6
:200F800068E670E087EA90E0AFDC60E087EA90E05ADC87EA90E01ADD41E050E068E670E029
:200FA00087EA90E011DD87EA90E0FEDB87FB882780F9C82F80E0D82F81E0C8278C2FDF9125
:200FC000CF910895CF92DF92EF92FF920F931F93CF93DF93EC0168E670E087EA90E084DC3C
:200FE00060E087EA90E02FDC87EA90E0EFDC47E050E068E670E087EA90E0E6DC87EA90E0A0
:20100000D3DB8F77982F92959F701AEF082F919F000D112487EA90E0C7DB9C013327A4E06F
:2010200035952795AA95E1F7F82E129FF00C112487EA90E0B9DB9C013327B4E03595279585
:20104000BA95E1F7E82E129FE00C112487EA90E0ABDB87EA90E0A8DB9C01332794E0359581
:2010600027959A95E1F7D82E129FD00C112487EA90E09ADB9C01332744E0359527954A950F
:20108000E1F7C82E129FC00C112487EA90E08CDB9C01332754E0359527955A95E1F7129F5F
:2010A000800D11248883C982DA82EB82FC820D83CE01DF91CF911F910F91FF90EF90DF90D5
:2010C000CF9008951F920F920FB60F9211242F933F938F939F93AF93BF9380916801909110
:2010E0006901A0916A01B0916B013091670126E0230F2D3720F40296A11DB11D05C029E86A
:20110000230F0396A11DB11D209367018093680190936901A0936A01B0936B0180916C0189
:2011200090916D01A0916E01B0916F010196A11DB11D80936C0190936D01A0936E01B093B6
:201140006F01BF91AF919F918F913F912F910F900FBE0F901F9018953FB7F89480916C0148
:2011600090916D01A0916E01B0916F0122B708B600FE05C02F3F19F00196A11DB11D3FBF9D
:201180006627782F892F9A2F620F711D811D911D43E0660F771F881F991F4A95D1F708957E
:2011A000CF92DF92EF92FF92CF93DF936B017C01D3DFEB01C114D104E104F10479F0E7D04C
:2011C000CBDF6C1B7D0B683E7340A0F381E0C81AD108E108F108C851DC4FECCFDF91CF919D
:2011E000FF90EF90DF90CF900895789483B7826083BF83B7816083BF89B7816089BF1EBC6C
:201200008EB582608EBD8EB581608EBD8FB581608FBD85B5846085BD85B5806485BD329AF2
:20122000319A3098379A1AB80895843039F0863049F0833051F48FB58F7702C08FB58F7DBB
:201240008FBD089585B58F7D85BD0895CF93DF9390E0FC01E05AFF4F2491FC01EC58FF4F73
:201260008491882349F190E0880F991FFC01E456FF4FA591B4918E569F4FFC01C591D4912B
:201280009FB7611108C0F8948C91209582238C93888182230AC0623051F4F8948C91322F43
:2012A000309583238C938881822B888304C0F8948C91822B8C939FBFDF91CF9108950F933D
:2012C0001F93CF93DF931F92CDB7DEB7282F30E0F901E45BFF4F8491F901E05AFF4F149194
:2012E000F901EC58FF4F04910023C1F0882319F069839BDF6981E02FF0E0EE0FFF1FEE56B7
:20130000FF4FA591B4919FB7F8948C91611103C01095812301C0812B8C939FBF0F90DF918E
:20132000CF911F910F910895CF93DF93282F30E0F901E45BFF4F8491F901E05AFF4FD491A2
:20134000F901EC58FF4FC491CC2389F081116DDFEC2FF0E0EE0FFF1FE857FF4FA591B49158
:201360002C912D2381E090E021F480E002C080E090E0DF91CF910895089537DFFDDF3AD77B
:20138000C0E0D0E0AFD92097E9F33AD6FBCF0895991B79E004C0991F961708F0961B881FE5
:2013A0007A95C9F780950895AA1BBB1B51E107C0AA1FBB1FA617B70710F0A61BB70B881FD0
:2013C000991F5A95A9F780959095BC01CD01089597FB072E16F4009406D077FD08D0E4DF1A
:2013E00007FC05D03EF4909581959F4F0895709561957F4F0895EE0FFF1F0590F491E02D75
:201400000994F894FFCF09000300040007000600050008000B000C000D000A000F0010005E
:2014200011000E0031353A34353A333800446563203138203230313800000000002304F741
:0A14400003CC03D403E703F6030016
:00000001FF
